:0200000480007A
:100000006F00C004732F2034930F8000630AFF0336
:10001000930F90006306FF03930FB0006302FF038A
:10002000170F0080130F0FFE63040F0067000F000F
:10003000732F203463540F006F004000136E9E53E3
:10004000171F00002320CFFD6FF09FFF732540F1A5
:100050006310050073251030635805000F00F00F82
:10006000130E100073000000130E00009702000032
:10007000938282F973905230735020307350303035
:1000800073504030970200809382C2F7638C020065
:10009000739052109302B01A739022307323203061
:1000A000E39E62F873500030970200009382420191
:1000B00073901234732540F17300203093000000D8
:1000C00093B10000930E0000130E20006392D1271D
:1000D0009300100093B11000930E0000130E300037
:1000E0006398D1259300300093B17000930E1000F7
:1000F000130E4000639ED1239300700093B1300033
:10010000930E0000130E50006394D123930000005F
:1001100093B10080930E1000130E6000639AD121FA
:10012000B700008093B10000930E0000130E700022
:100130006390D121B700008093B10080930E10002E
:10014000130E80006396D11F9300000093B1F07FDF
:10015000930E1000130E9000639CD11DB700008019
:100160009380F0FF93B10000930E0000130EA000E7
:100170006390D11DB70000809380F0FF93B1F07FB2
:10018000930E0000130EB0006394D11BB7000080E3
:1001900093B1F07F930E0000130EC000639AD11943
:1001A000B70000809380F0FF93B10080930E1000A1
:1001B000130ED000639ED1179300000093B1F0FF9F
:1001C000930E1000130EE0006394D1179300F0FF1C
:1001D00093B11000930E0000130EF000639AD11536
:1001E0009300F0FF93B1F0FF930E0000130E000197
:1001F0006390D1159300B00093B0D000930E10001F
:10020000130E10016396D013130200009300F00048
:1002100093B1A00013830100130212009302200087
:10022000E31652FE930E0000130E20016312D31149
:10023000130200009300A00093B10001130000001E
:10024000138301001302120093022000E31452FEF4
:10025000930E1000130E3001631CD30D1302000027
:100260009300000193B19000130000001300000000
:10027000138301001302120093022000E31252FEC6
:10028000930E0000130E40016314D30B1302000001
:100290009300B00093B1F00013021200930220000B
:1002A000E31852FE930E1000130E50016392D10911
:1002B00013020000930010011300000093B18000AE
:1002C0001302120093022000E31652FE930E000068
:1002D000130E6001639ED105130200009300C0005D
:1002E000130000001300000093B1E000130212009D
:1002F00093022000E31452FE930E1000130E7001BF
:100300006398D1039330F0FF930E1000130E800119
:100310006390D003B700FF009380F00F13B0F0FF9D
:10032000930E0000130E90016314D001631CC001F2
:100330000F00F00F63000E00131E1E00136E1E0050
:10034000730000000F00F00F130E10007300000088
:10035000731000C00000000000000000000000005A
:10036000000000000000000000000000000000008D
:10037000000000000000000000000000000000007D
:040380000000000079
:1010000000000000000000000000000000000000E0
:1010100000000000000000000000000000000000D0
:1010200000000000000000000000000000000000C0
:1010300000000000000000000000000000000000B0
:081040000000000000000000A8
:040000058000200057
:00000001FF
